:10800000000001208DDB000099BA000099BA000041
:1080100099BA000099BA000099BA00000000000067
:1080200000000000000000000000000099BA0000FD
:1080300099BA00000000000099BA0000698F0000A2
:1080400099BA000099BA000099BA000099BA0000E4
:1080500099BA000099BA000099BA000099BA0000D4
:1080600099BA000099BA000099BA000099BA0000C4
:1080700099BA000099BA000099BA000099BA0000B4
:1080800099BA000099BA000099BA000099BA0000A4
:1080900099BA000099BA000099BA000099BA000094
:1080A00099BA000099BA000099BA000099BA000084
:1080B00099BA000099BA000099BA000099BA000074
:1080C00099BA000099BA000099BA000099BA000064
:1080D00099BA000099BA000099BA000099BA000054
:1080E00099BA000099BA000099BA000099BA000044
:1080F00099BA000099BA000099BA000099BA000034
:1081000099BA000099BA000099BA000099BA000023
:1081100099BA0000B590000099BA000099BA000021
:1081200099BA000099BA000099BA000099BA000003
:1081300099BA000099BA000099BA000099BA0000F3
:1081400099BA000099BA000099BA000099BA0000E3
:1081500099BA000099BA000099BA000099BA0000D3
:1081600099BA0000E5CC000099BA000099BA000065
:1081700099BA000099BA000099BA000099BA0000B3
:1081800099BA000099BA000099BA000099BA0000A3
:1081900099BA000099BA000099BA000099BA000093
:1081A00099BA000099BA000099BA000099BA000083
:0C81B00099BA000099BA000099BA0000CA
:10840000FFFFFFFFFFFFFFFFFFFFFFFF7EF9FFFF03
:1084100010B5054C237833B9044B13B10448AFF3BE
:1084200000800123237010BD0006FF1F0000000024
:1084300050DF00000C4B43B10C480D4910B5AFF3B1
:1084400000800C48036823B910BD0A48036833B99B
:108450007047094B002BF7D0BDE810401847064B7A
:10846000002BF5D0184700BF0000000050DF0000CF
:108470000406FF1F2C05FF1F0000000080F3118879
:1084800070472F4B41F238015A5842F478525A50F3
:108490002C4A927902F00C020C2A4FD041F244028D
:1084A0002949995003F558339A78110748BF9A78AB
:1084B000264944BF42F008029A70214B41F244021F
:1084C000995041F204015A5842F4803242F0C002FD
:1084D0005A501A6842F440221A6003F5E833242205
:1084E0005A701B4A80211170A2221A70DA7802F0A9
:1084F0001F02DA7003221A7100225A719A799207C8
:10850000FCD59A79D006FCD40E4B19469A7902F024
:108510000C02082AFAD140225A718B7903F00C031D
:10852000082BFAD1074B1A4699794906FCD5222126
:108530001970937903F00C030C2BFAD1704700BF2C
:1085400000700440004006400000330100001301A9
:1085500000500640174B5A7902F0E0025A711A791E
:1085600002F0F8021A71144A136843F0040313600E
:10857000124A136823F0784323F001031360104B71
:108580001A7802F08C0242F050021A705A7802F007
:108590009C0242F040025A709A7802F0E6029A7009
:1085A000084A00231370084A82F8493383F311887C
:1085B000704700BF00F007404080044000D00040FA
:1085C00000D0074000E0074000E100E010B51420B3
:1085D00000F084FC1228074C09D1152000F07EFC25
:1085E000342804D1102000F079FC207010BD08233D
:1085F000237010BD1C06FF1F2DE9F041C14DC24F75
:108600006E78032E88B040F0A2803B784BBBBF4E03
:10861000737834781C44F37903341C44B3791C44D4
:1086200073791C44337902201C4400F001FD0120C1
:1086300000F0FEFC307800F0FBFC707800F0F8FCF5
:10864000F07900F0F5FCB07900F0F2FC707900F000
:10865000EFFCE4B2307900F0EBFC204600F0E8FCDF
:1086600009E0012B07D1AA4E0024305D013400F04F
:10867000DFFC092CF9D100236B703B70AB7813B190
:10868000012000F077FD0DF1070000F0E9FC044641
:10869000002800F0D78000F0FBFC08B10023EB704D
:1086A000EA789DF80710531CDBB22A44092BEB70C3
:1086B000117121D12A790023012AEB701CD1954830
:1086C0001A46195C01330A44082BD2B2F9D12B7B2C
:1086D000934240F0B580904B6A791A70AA795A702B
:1086E000EA799A702A7A9A716A7A5A71AA7A1A7110
:1086F000EA7ADA7003236B706B7803F0FB02032ACB
:1087000002D0052B40F03581834ADFF800821378D0
:1087100088F80130642188F80010472BD2F8031044
:10872000C8F804104446164600F0328100F2C880B2
:10873000422B00F0218100F2B8800A2B00F00C815E
:1087400000F2AB80092B00F0FB80022348E2042EEC
:1087500021D16E4C00234FF001080220637063604A
:1087600084F8008000F064FC404600F061FC207852
:1087700000F05EFC607800F05BFCE07900F058FCF3
:10878000A07900F055FC607900F052FC207900F0EF
:108790004FFC304662E7072E33D13B7805A833BB48
:1087A0005A4A137892F801E0D6798DF8163073445E
:1087B000947951798DF819400333334412798DF847
:1087C0001A101C444FF0020C21448DF814C08DF88F
:1087D0001B204FF0010C0A448DF815C08DF817E0EE
:1087E0008DF818608DF81C2000F038FD43E7012B50
:1087F000FAD1474900235A5CC2540133092BFAD1FC
:10880000F2E7082E7FF437AF4049002301224B7076
:108810004B600A708DF8173002218DF818308DF8F2
:1088200019308DF81A308DF81B3004238DF8141090
:108830008DF815208DF816208DF81C3005A8D3E78B
:10884000042358E702AE304600F0F7FC00283FF45E
:1088500053AF2346F25C01331444082BE4B2F9D140
:108860009DF81020A2427FF446AF2B4B9DF80920C3
:108870001A709DF80A205A709DF80B209A709DF886
:108880000C209A719DF80D205A719DF80E201A71D6
:108890009DF80F20DA7007232DE7402B67D0412B7E
:1088A0007FF453AF00F023FA63E0442B6AD066D321
:1088B000452B6AD0462B7FF448AF00F042FA58E0CF
:1088C000932B00F0118129D88F2B7FD00AD8882BC9
:1088D0007FF43BAF5378012B6DD05CD3052B39D19E
:1088E000012342E0902B00F00C81922B7FF42DAFFE
:1088F0009378002B00F0A380FF2B00F0B3800423BB
:108900006EE100BF1C06FF1F1F0BFF1F2C0BFF1F7C
:10891000200BFF1F2006FF1F180BFF1F952B00F0D9
:10892000E980C0F0B280F22B00F05C81FF2B7FF475
:108930000CAF40F2D24399421BD10123AB7018E037
:108940005378013B032B05D8DFE803F01313021320
:1089500001290ED9032343E15378013B032BF9D8B6
:10896000DFE803F0020202560023636001E000F03A
:10897000BDF908B0BDE8F08100F0CEF9F9E700F0EC
:10898000DDF9F6E700F0DBF9F3E700F0D9F9F0E7FD
:1089900000F0D8F9EDE70123C04A3B7002231370C1
:1089A000BF4B196800230139013311F8010FD0546E
:1089B000082BF9D1DDE700220C2188F8072088F880
:1089C000061088F8053088F80420D2E75378042B85
:1089D000C0D8DFE803F0031811111C00142000F0C8
:1089E0007DFA12280CD1152000F078FA342807D12E
:1089F000102000F073FA2870022363712B7810E0C6
:108A000008232B70F8E7F3782B70022208E071B985
:108A10002B78082BF9D0A3F11A02012AF5D90622E6
:108A2000627123710423E3710023A371A1E7F3783A
:108A3000082BE1D01A3B012BDED90623DDE7507865
:108A4000831FDBB21E2B00F21181964A22FA03F338
:108A5000DA0700F10E81392800F00B81000102F0E5
:108A6000B9FA86E798F804306B74507898F80530B6
:108A7000AB7498F80630EB74082298F807308A49EE
:108A80002B75000102F0E1FA73E793782BB1FF2B0D
:108A900017D0042388F800306BE75078831FDBB2CF
:108AA0001E2B00F2EF807F4A22FA03F3DB0700F16E
:108AB000EC80392800F0E980000102F0A9FB606039
:108AC00057E7507879490822000102F0E8FB2B7F34
:108AD00088F80730EB7E88F80630AB7E88F80530E2
:108AE0006B7E88F8043044E7D178B2F8010002F0D8
:108AF00011FC3EE7B2F8010002F0C7FCC8F8040020
:108B000037E75578012D3ED032D3022D7FF422AFC6
:108B10004FF4A06002F08DFCC10760D5012140F246
:108B2000015002F0F7FB40F2025002F0AEFC0204EA
:108B3000F9D4D6F8031040F20450091402F03EFCB8
:108B4000D6F803104FF4A16089B202F037FC40F26E
:108B5000025002F09AFC40F4007140F2025002F020
:108B600000FC40F2025002F090FC0304F9D431E022
:108B70005221412002F0CEFB4521412002F0CAFBE8
:108B800053214120B3E74FF4A06002F052FCC70725
:108B900025D5294640F2015002F0BCFB40F20250BC
:108BA00002F073FC0504F9D4D6F8031040F2045027
:108BB00002F004FC40F2025002F067FC40F48071C5
:108BC00040F2025002F0CDFB40F2025002F05DFC98
:108BD0000004F9D44FF4A16002F08DFC6FE7062386
:108BE0002370C6E65378812B7FF489AE9378922B5D
:108BF0007FF485AE9379A32B7FF481AE5379B42BA8
:108C00007FF47DAE1379C52B7FF479AED378D62B64
:108C10007FF475AE00F025FB00F0D0F9044600F0BB
:108C2000CDF9001B0028B8BF4042B0F57A7FF6DBD3
:108C300000F09EFA1E4B00221A604FF0FF32C3F87C
:108C40007021C3F87022C3F87421C3F87422C3F8EA
:108C50007821C3F87822C3F87C21C3F87C22154B15
:108C6000154A1A60012000F085FA82E637287FF461
:108C7000F2AE23796B736379AB73A379EB73E3790A
:108C80002B7476E637287FF414AF2B7EE371EB7DEF
:108C9000A371AB7D63716B7D23716AE6200BFF1FAF
:108CA0000800FF1F030000582906FF1F3106FF1FA1
:108CB00010E000E00000FF1F78563412704710B536
:108CC000084C00F07BF92368C01A0028B8BF404266
:108CD000FA2805DD044B0422DA6000F06FF9206009
:108CE00010BD00BF3C06FF1F00F00F407047074B50
:108CF0005A78012A05D104220549D3F8030000F06F
:108D00000AB9044B03221A70704700BF180BFF1FEB
:108D1000300BFF1F2C0BFF1F064B5A78012A04D182
:108D20009978D3F8030000F00FB8034B03221A70B0
:108D3000704700BF180BFF1F2C0BFF1F70477047B9
:108D400070477047704700BF38B5012204460D4692
:108D50004FF48270062100F0F3FA002205214FF44F
:108D6000827000F0EDFA012200214FF4827000F0D1
:108D7000E7FA8207F1D5002202214FF4827000F059
:108D8000DFFA0022C4F307214FF4827000F0D8FA12
:108D90000022E1B24FF4827000F0D2FA012229469B
:108DA0004FF4827000F0CCFA002205214FF482705B
:108DB00000F0C6FA012200214FF4827000F0C0FAE0
:108DC000C307F1D438BD2DE9F8430446884616465A
:108DD000062101224FF4827000F0B2FA0022052130
:108DE0004FF4827000F0ACFA012200214FF482703F
:108DF00000F0A6FA8507F1D5002202214FF4827017
:108E000000F09EFA0022C4F307214FF4827000F0B4
:108E100097FA0022E1B24FF4827000F091FA002537
:108E2000771EB5420FD1002205214FF4827000F069
:108E300087FA012200214FF4827000F081FAC30703
:108E4000F1D4BDE8F883013414F03F0918F8051097
:108E500042D0781B424242414FF4827000F070FAD7
:108E6000B9F1000F36D1BD4234D2002205214FF4B2
:108E7000827000F065FA002101224FF4827000F048
:108E80005FFAC107F1D4012206214FF4827000F08D
:108E900057FA002205214FF4827000F051FA0122A6
:108EA00000214FF4827000F04BFA8207F1D50022C6
:108EB00002214FF4827000F043FA0022C4F307212C
:108EC0004FF4827000F03CFA0022E1B24FF482705D
:108ED00000F036FA0135A4E70122BDE710B5002203
:108EE000044603214FF4827000F02AFAC4F30721EC
:108EF00000224FF4827000F023FAE1B200224FF416
:108F0000827000F01DFA012200214FF48270BDE84A
:108F1000104000F015BAF8B504460E461546032178
:108F200000224FF4827000F00BFAC4F307210022F4
:108F30004FF4827000F004FAE1B200224FF4827024
:108F400000F0FEF977193446013DBC4200D1F8BD6E
:108F5000A21BAB1A5A425A4100214FF4827000F012
:108F6000EFF904F8010BF0E70D4A6846136820F0AA
:108F700007018D46013301B513600A4B1A68092AAF
:108F800088BF0022BDE8014085BF1A605A681A6890
:108F9000013296BF01325A601A608546704700BFA1
:108FA000340BFF1F4006FF1F034B4FF416525A604D
:108FB00007221A60704700BF10E000E0014B5868BC
:108FC000704700BF4006FF1F1449154B41F22802AD
:108FD000072888BF002010B553F82030114CB4FB8F
:108FE000F3F48B5843F480638B500F4B4FF4407273
:108FF0009A633520DA6302F067FD0C4B0022DA70C9
:109000009A709A71DA725A71C4F30422E4B21A7037
:109010005C70DA7842F02C02DA7010BD0070044007
:10902000F0DD0000C0C62D0000B0044000A00E40DE
:10903000094A136851680133202B08BF00238B4273
:1090400008D01168114408721360044AD37843F0C1
:109050008003D370704700BF4806FF1F00A00E407A
:109060000A4B996ADA6A91420DD09A6A511C1A44E5
:10907000996292F8302002709A6A202A01D1002267
:109080009A62012070470020704700BF4806FF1F0A
:10909000044B1A7802F0FF0012B100221A7001206E
:1090A000704700BF380BFF1F014B1865704700BFAA
:1090B0004806FF1F684620F007018D4611B5264C73
:1090C0002179C9B2880615D5244BDA6A986A01322B
:1090D000202A08BF0022824206D0D86AE4791844C8
:1090E000E4B280F83040DA621D4A052010601A6D43
:1090F0001C4B1A604A0608D51B4B4FF400329A608D
:10910000154AD37803F0BF03D3700B061BD5154B5C
:109110001868C0B9114B19685A68914217D0124AA1
:109120004FF4003151605A68511C1A445960117A49
:10913000094AC9B2D1715968202908BF5860D3784B
:1091400043F04003D370BDE8114085467047024AA2
:10915000D37803F07F03F5E700A00E404806FF1F19
:109160003C0BFF1F400BFF1F00F00F4062B6704723
:1091700072B670474FF0E02318B1034AC3F80C2DC4
:109180007047024AFAE700BF0400FA050100FA0539
:109190001F4A4FF48073536093605361136302F569
:1091A000362241F2060191602021516041F22601F0
:1091B0005161A2F535224FF48021936402F53522E6
:1091C00040325160516113490A7842F080020A70BE
:1091D000A1F5F03141F20402885820F0E0008850F7
:1091E000885840F0C00088500B4A4FF4A061D1600D
:1091F00013601361136202F53422803240F21111C0
:1092000051615160054A1360054B00225A61704755
:10921000009004400050064000B0044000C00440EC
:10922000C0F00F4008B504F081FB02F03FFE02F0F1
:10923000EFFDBDE8084004F0FBBB38B5054602F081
:109240003DFD082808D900242819013402F0B6FD94
:10925000092CF9D1012038BD002038BD092102F0C8
:109260004DBD002002F0DABF2F4B41F23C0170B53A
:109270005A582E4C2E4E2F4D42F440525A5041F225
:10928000300101205A5842F480525A50A3F5D83385
:1092900018601A6822431A60274ADA601A61DA6A8B
:1092A00042F08052DA621A6822F001021A601A68EB
:1092B00022F000621A6003F5F8334FF400725A612D
:1092C0009A61DA61A3F5F0331860196821431960D7
:1092D000DE601D61D96A41F08051D962196821F0C0
:1092E00001011960196821F00061196003F5FE237E
:1092F00012498A62CA620A644A6418601868204384
:109300001860DE601D61D86A40F08050D86218682D
:1093100020F001001860186820F0006018604A65AD
:109320008A65CA6570BD00BF00700440000C1F80D4
:109330000400513E0400F13E0300013E00A0044041
:10934000B0F5827F30B507D040F20123984245D076
:1093500040F20113984264D10304334C1AB3B0F5C0
:10936000827F02BF314A4FF48025956003F47C135D
:1093700041F000612C4A194361631346D16A002908
:10938000FCDADA6AD100FCD5996BDA6AB0F5827F33
:1093900042F01042C9B2DA6203D1244B4FF480226A
:1093A0005A60084630BDB0F5827F03F47C1308BFD5
:1093B0001E4A41F0004141EA030108BF4FF48020FA
:1093C000194B08BF90606163DA6A002AFCDA996B76
:1093D000DA6A42F01042C9B2DA62E2E7144C154B85
:1093E0000120A060A2B141F0006141F480315963D5
:1093F000DA6A002AFCDA0F4BDA6AD200FCD5996BE4
:10940000DA6A42F01042DA620123C9B26360C8E747
:1094100041F0004141F480315963DA6A002AFCDAF4
:10942000D5E70021BDE700BF00D0024040F00F406B
:1094300080F00F4000C00A4070477047002070471E
:1094400010B5064C204602F011FB054B1A88054B5F
:1094500020461988BDE8104001F0AEBB8C0BFF1F01
:10946000FC0BFF1F100CFF1F10B5064B064C1A8893
:10947000064B2046198801F037FB2046BDE8104016
:1094800002F0FABAEE0BFF1F460BFF1FF40BFF1F93
:1094900070B4534B53481B78534943B101230370B5
:1094A00000230B700978007870BC01F021BC4F4B91
:1094B0001A88013292B2322A1A8005D0642A03D067
:1094C000962A01D0C82AEDD1494C2578494C05F09F
:1094D0000F05013D072D45D8DFE805F04404423E65
:1094E00044444440402525702578AC0601D4C82A60
:1094F00012D115F01F0218BF52009C781CBF02F158
:10950000FF32D2B2AC422FD02E064CBF0022012235
:10951000027001229A809D70374A1578AA0602D4FB
:109520001A88C82A12D115F01F0218BF52009C7960
:109530001CBF02F1FF32D2B2AC4233D02E064CBF78
:10954000002201220A7001221A819D711A88C82AFC
:1095500004BF00221A80A5E74125C4E70125C2E720
:109560006025C0E70025BEE76C0617D50478B4FA7D
:1095700084F464090470002ACDD09C880134A4B21C
:1095800094429C80C7D92E0602F104024CBF0126EA
:109590000026A2420670BEDA0022BBE705F00102F7
:1095A0000270B8E76C0617D50C78B4FA84F4640935
:1095B0000C70002AC9D01C890134A4B294421C81C9
:1095C000C3D92E0602F104024CBF01260026A24296
:1095D0000E70BADA0022B7E705F001020A70B4E7AC
:1095E000060CFF1FD00BFF1F8A0BFF1F9C06FF1FDF
:1095F000ED0BFF1FF60BFF1F0E0CFF1F064B1B781A
:109600003BB1064AB2F90030002BC4BF03F1FF336F
:109610001380FFF73DBF00BFFA0BFF1F020CFF1FB7
:1096200037B502AC002501F065F844F8045D04226A
:1096300020464FF4A06101F01EFA019B204623F45E
:109640007F4304224FF4A061019301F084FA034B9D
:10965000012228469A7203B030BD00BF9C06FF1F4E
:1096600008B51C4B9B7A002B32D01B4B1B7883B167
:109670001A4B1B78CBB101F079FB092803D9FFF70E
:10968000BDFF01F079FB01F091F8BDE8084000F062
:1096900073BF01F0C0FA420510D5104B01221A70B9
:1096A0000F4B1B780BB1FFF7DFFE02F0EBF90D4B10
:1096B0001B78002BDFD0FFF7C3FEDCE70A4B1B88CB
:1096C000002BF2D1030542BF044B01221A70ECE7D4
:1096D00008BD00BF9C06FF1F0B0CFF1F000CFF1FE7
:1096E000060CFF1F0A0CFF1FEE0BFF1F02F0CAB98A
:1096F0002DE9F04F85B0884601904FF4A06103A892
:1097000092460222994601F0B6F9022240F2025135
:109710000DF10E0001F0AFF9BDF80C4014F001049A
:1097200000F08480B9F1000F06D1BDF80E3013F0BF
:10973000400F14BF042402244FF4807302224FF41C
:10974000A06103A8ADF80C3001F005FA00264FEA3D
:10975000440B0A27354645450DD30024002303A8B2
:1097600002224FF4A061ADF80C3001F0F4F920466C
:1097700005B0BDE8F08F042240F204510DEB020069
:1097800001F0E9F9B9F1000F34D14FF480730222EE
:1097900040F202510DF10E00ADF80E3001F0DBF990
:1097A000022240F202510DF10E0001F064F9BDF900
:1097B0000E30002BF4DB022240F202510DF10E00BC
:1097C00001F059F9BDF80E3013F4F04F1CD09B0492
:1097D00000D46FBB013FFFB2BDF80E3003F4F0437D
:1097E0002BB9019B264423440193B6B20A27254492
:1097F000ADB2B0E702224FF4A1610AEB450001F0DF
:10980000AAF94FF40073C2E7B9F1000FE4D133199C
:109810004345C3BFA8EB0602520092B25A464FF42A
:10982000A1610AEB450001F026F9D5E7502495E740
:10983000512493E710B586B0FF23ADF8063002AC93
:109840000023224607211846FFF752FF00BBBDF850
:109850000630225C5340082213F0800F02F1FF32E1
:109860004FEA430318BF83F0070392B29BB2002A6A
:10987000F2D101300E28ECD106AADBB222F8123D5B
:10988000012319460720FFF733FF002808BF2020D7
:1098900006B010BD034A00231380034A1360034A35
:1098A00013607047D80BFF1FDC0BFF1FE00BFF1F7F
:1098B0000188072938B5044640F2F8800389083941
:1098C000013B89B2052B00F2B680DFE803F00345C7
:1098D000566C8D977A4B1D88002D40F0EC8000F17E
:1098E0001002C368104600F0EBFF764B01221A60AD
:1098F000754B1D60754B186047F69573984200F2E2
:109900008B80704B1B68E36000F108032380704B71
:109910001B880E3B03229842694B22810CBF012217
:1099200004221A806B4B1D78002D00F0B7806A4B23
:1099300062791978490704BF01211970197802F07A
:109940000F02627142EA0112627101312046197000
:1099500001F006FF002038BD594B1D88002D40F056
:10996000AA80C268103000F0DDFF47F6FD730028C2
:1099700008BF1846534B1D60BEE7514B1B8823F0B0
:1099800004039BB2022B40F096804E4BC2681B68CA
:109990009A4240F08D80103001F002F80028ABD1DF
:1099A00047F6FD704FE0464B1B88012B0FD1474D0A
:1099B00000F11001286801F025F8434A2B68136074
:1099C000404A03442B6013680133136094E747F661
:1099D000FE7048F20402042B18BF1046050442D45E
:1099E000374B0020188038BD354B1B88002B62D0C8
:1099F000C06801F02BF847F6FF70EFE7304B1B888B
:109A0000012B01D0042B56D12F4BA089196804F1EA
:109A1000100201F017F86FE747F6FA7398420CD876
:109A200006232381A0F5FF4000237A38E381082331
:109A3000A081238076E748F20400A0F5FF437C3B39
:109A40009BB2012BCAD81F4A1368E360591C082334
:109A50001160238047F6FD730422984222811BD1B6
:109A60000222174B5DE70523238108232380E06052
:109A7000002303F0FE022244128A12F0FF0F04D0EA
:109A800012F47F4F04D10133DBB20933238003E0AA
:109A90000233DBB2202BECD10022E2E7402120464A
:109AA00001F018FF50B10D4B1C6053E7062038BD84
:109AB00048F2050092E748F204008FE738BD00BF86
:109AC000D80BFF1FDC0BFF1FE40BFF1FD40BFF1F86
:109AD0004413FF1F040CFF1F3813FF1FE00BFF1F71
:109AE00010B5044C206820B1002101F0F3FE0023E2
:109AF000236010BDE00BFF1F5C4B1B88B3F5405F7C
:109B000073B50546C0F0B080002001F021F98379DB
:109B1000DE0701D41624A4E0037903F00C02042A22
:109B2000F8D19C07F6D54388223B9BB2DE2BF1D8B7
:109B30000388A3F580539BB2B3F5005FEAD80120F8
:109B400001F006F98379DB07E4D5037913F00C04FF
:109B5000E0D19907DED54388223B9BB2DE2BD9D8D2
:109B60000388A3F580539BB2B3F5005FD2D8032DD1
:109B700026D93F4E01230320337001F0E9F88279A2
:109B80004388D20740D59BB13A4A12889A420FD1F6
:109B9000442A0DD8027912F00C0F09D136490388F6
:109BA0000978022906D1A3F58053B3F5005F05D9E2
:109BB0001E2456E0314909889942F9D1900720D4F2
:109BC000022D37D9022001F0C3F882794388D107EA
:109BD00035D5A3B12A4A12889A4210D1442A0ED808
:109BE000037903F00C02042A09D123490288097879
:109BF000022910D1A2F58052B2F5005F0FD91D24C1
:109C00002FE000233370DDE7002BD1D1194B1B88E7
:109C1000002BCDD1D4E71B4909889142EFD113F035
:109C20004001194A18BF012111709A0702D5104B43
:109C300000221A7000238DF80730144E0EE0002B1E
:109C4000DDD10F4B1B88002BD9D1F3E7284601F05B
:109C50007FF8013583798DF80730EDB23378AB4268
:109C6000F4D8204602B070BD1424FAE7FE0BFF1FA3
:109C7000E80BFF1FFC0BFF1FED0BFF1F100CFF1F5E
:109C8000EE0BFF1FF40BFF1F0C0CFF1F0D0CFF1F33
:109C90002DE9F3415F4A604E604C614D0023022084
:109CA0001370ADF80430ADF80630338001F050F891
:109CB000038823800379032013F0020F0CBF4FF0B9
:109CC00003084FF0010801F043F8564A0388138057
:109CD0000279B5F800E012F0020F534A0CBF0321DD
:109CE000012117880EFB0131B94205DD4F4A128868
:109CF0003A449342C0F285804D4A1088814204DD87
:109D00004C4A118801448B427BDB21884A4C2288D3
:109D100008FB0212974206DADFF810C1BCF800C057
:109D20006744B9426FDB904204DA424F3F883844BF
:109D3000814268DB934202DA7344994263DB012279
:109D400040F681110DF1030000F095FE9DF80330FF
:109D500013F0090F59D1394B1B78002B57D0384BD2
:109D60001B782BB12388002B3AD04FF480633380CB
:109D700002224FF484610DF1060000F07CFE23887E
:109D8000304E002B35D0BDF8063093B302224FF48D
:109D9000806101A800F06FFEBDF8043033B3BDF858
:109DA0000620023346F2A71103FB021346F2A81263
:109DB000B3FBF2F333803288234B1B78EAB9F3B953
:109DC000238813B1022000F0ABFF2B8813B10320CE
:109DD00000F0A6FFFFF734FB002002B0BDE8F081E1
:109DE0002B88002BC4D04FF40063C0E7ADF80630D9
:109DF000E0E70023ADF80430DCE7002BE0D11F20C2
:109E0000EBE71E20E9E71D20E7E73020E5E7292002
:109E1000E3E700BF000CFF1FF80BFF1FF40BFF1F51
:109E2000FC0BFF1F100CFF1F4E13FF1F4413FF1FDF
:109E30003C13FF1F5613FF1FEE0BFF1FE80BFF1F06
:109E40000B0CFF1F080CFF1F0C0CFF1F024B187898
:109E500008B1024B18887047F20BFF1FF00BFF1F71
:109E6000024A00231370024A13707047000CFF1F50
:109E7000060CFF1F08B50B4B1B8813B1022000F026
:109E800038FF094B1B8813B1032000F032FF074A4B
:109E900000231370064A1370064A1370064A1370A3
:109EA00008BD00BFEE0BFF1FFC0BFF1F000CFF1FC8
:109EB0000C0CFF1F0A0CFF1FA706FF1F73B51C4DDC
:109EC000ADF806102B7883424FF6FF7318BF287049
:109ED000994206460C4606D002224FF49A710DF1C3
:109EE000060000F038FE2B78ADF8063002224FF461
:109EF00098710DF1060000F02EFE0E4A0CB1F1062D
:109F000003D40023137002B070BDA4F11A0399B2F8
:109F100018299DBF084BCB40DB430123DB0701D44D
:109F20004123EFE71B2C0CBF42234023EAE700BF8D
:109F3000ED0BFF1F0E0CFF1F010008012DE9F04F74
:109F4000C34FC44DC44C85B04FF6FF733B80012214
:109F500010F01003029301912A7000F00F00237893
:109F600033D023F01003237002922378DFF80883A4
:109F7000C6B206EB031303F0FF0BBBF1440F3AD05C
:109F800032D8BBF1220F3FD028D8BBF1120F3BD003
:109F9000B24903914FF0000ABBF1310FA1F800A0C4
:109FA00000F0288100F2A580BBF1180F58D000F214
:109FB0008F80BBF1120F00F036814AD8BBF1110F30
:109FC00000F08F814FF012094CE0DA0602D501282B
:109FD00040F00D8103F00F032370C6E7BBF1240F9F
:109FE0001BD0BBF1420FD2E7BBF1820F0CD005D8DA
:109FF000BBF1480FCCD19A4A107806E0BBF1840F30
:10A00000F9D0BBF1880FF5E70220FFF775FD1FFAC5
:10A0100080F9B9F1000F07D1BAE79249924801F0EF
:10A0200020FD81460028E6D02278042A00F07881BD
:10A03000082A00F07181022A40F07981B9F1160FE7
:10A0400040F0738101F02AFB01F001FD0123237030
:10A0500008E0BBF1130F00F09680BBF1140FB1D1F3
:10A060004FF01109207800F00F039E4200F0898123
:10A07000B9F1000F03D1019B002B00F07E8130432A
:10A0800003070ED5794B1B781BB101F0E8FCFFF7F5
:10A09000E7FE744B1B88002B00F06481022000F067
:10A0A00028FEB9F1000F00F064812378082B04BF6B
:10A0B00004232370237843F01003237000232078B7
:10A0C00088F80030494605B0BDE8F04FFFF7F6BE0E
:10A0D000BBF1230FC4D005D8BBF1210F21D0BBF1B8
:10A0E000220F6DE7BBF1240F00F0C880BBF1280FF1
:10A0F000B5E7BBF1480F00F0D28020D8BBF1420F8A
:10A1000032D016D8BBF1410F7FF45CAF01F0A3FC55
:10A110008146FFF7AFFE00232B70B9F1000F40F02E
:10A120005D8101F0BBFA01F092FC4FF0210B8146FA
:10A130006EE0BBF1430F93D0BBF1440F40E7BBF19E
:10A14000830F8DD018D8BBF1810F00F0C080BBF118
:10A15000820F7FF437AF01F082FC8146FFF780FE6B
:10A1600085F800A0002853D101F075FCFFF782FEAE
:10A1700000212970894675E7BBF1840F00F09F80AC
:10A18000BBF1880F1CE7DFF8ECB0012302208BF84D
:10A190000030FFF7B1FC20B18BF800A04FF015099B
:10A1A00060E701F04DFA1FFA80F9B9F1000F40F0B5
:10A1B000EC8085F8009001F048FC8146002840F0D2
:10A1C000E4802B4B01221A700320FFF735F9B9F117
:10A1D000FF0F7FF447AF0123039A88F80030132361
:10A1E00013804FF4FA633B803B88323B3B8005B0E1
:10A1F000BDE8F08F1F4801780029BBD080F800A08F
:10A200000220FFF779FC01F049FA01F020FC8146B9
:10A21000B9F1FF0F7FF426AF039B012288F80020DD
:10A22000A3F800B096E001F00BFA1FFA80F9B9F13B
:10A23000000F40F0B58085F8009001F006FC8146E3
:10A24000002840F0AD800A4B01221A700AE700BFD7
:10A25000020CFF1FEC0BFF1FED0BFF1FEA0BFF1F94
:10A260000D0CFF1FEE0BFF1FFC0BFF1F060CFF1F4B
:10A270003A13FF1F040CFF1FFA0BFF1FFFF708FD27
:10A280008146002840F096802870564801F0E1FB96
:10A290008146002840F08E800122534BD5E7FFF71E
:10A2A000D5FD8146002840F08F80287001F0D5FB55
:10A2B0008146002840F0888001224C4BC5E701F020
:10A2C000CEFBD146FFF7CCFD85F800A0CAE601F031
:10A2D000C6FB8146FFF7C4FD85F800A0002897D192
:10A2E00014E7029B13B1584601F0AEFB404B1B78BC
:10A2F0004BB9237813F00C0F05D03E4B1B882BB1C4
:10A30000022000F00DFD4FF0FE09ABE63A4B1B8832
:10A31000002BF8D00320F4E701F0A1FBFFF7A0FD2C
:10A3200001F099FBFFF7A6FD88E602222270B9F141
:10A33000FF0F7FF497AE012288F800202F4ABBF16F
:10A34000240FA2F800B00AD006D8ABF11203012BFB
:10A350007FF647AFC82346E7BBF1480FFAD142F278
:10A36000283340E7244B1B88002B3FF49AAE032090
:10A3700095E6019B0BB146F010062670DDF80490BF
:10A380009CE6002188F800109DE6B9F1FF0F3FF42C
:10A390001BAF2B780BB901F05AFB01F07FF913E7E3
:10A3A000B9F1FF0FC7D02B780BB901F050FB01F0CA
:10A3B00075F957E6B9F1FF0FBDD02B780BB901F055
:10A3C0004AFBFFF757FD4DE6B9F1FF0FB3D02B78ED
:10A3D0000BB901F044FBFFF743FD43E64FF0410B9F
:10A3E00016E700BFF80BFF1F0A0CFF1F060CFF1F2C
:10A3F000F20BFF1FEE0BFF1FFC0BFF1FEA0BFF1FF3
:10A4000038B5514D2B788BB1504B514CB3F90030CE
:10A41000002B3BD12388242BC3F307142ED006D85E
:10A42000123B012B10D9002C40F08A8038BD482BFC
:10A43000F9D1484B1B780BB901F011FBFFF710FD68
:10A440001B20002C77D138BD424B1B780BB901F093
:10A45000FEFA01F023F9404B1B78002B6ED03F4BE6
:10A460001888002CE2D000232B7008B144F01004AF
:10A4700001462046BDE83840FFF720BD354B1B782C
:10A480000BB901F0E8FAFFF7F5FCE4E72388242B89
:10A490001FD003D8123B012B03D938BD482B2FD036
:10A4A00038BD2C4B1A78002AC0D000221A7001F057
:10A4B000CCFA30B92A4B247801221A7004F00F0428
:10A4C000B1E7FF28B2D001F0C2FABDE8384001F090
:10A4D000E5B8204B1A78002AA8D0002221481A702B
:10A4E00001F0B7FA20B9204B01221A700424BAE710
:10A4F000FF289BD001F0AFFABDE83840FFF7BABCA7
:10A50000144B1B78002B91D0184B1B881BB1184B98
:10A510001B78002B8AD001F0A0FA20B9154B01223C
:10A520001A7008249FE7FF2880D001F098FABDE850
:10A530003840FFF795BC00232B7097E7012080E798
:10A540000020287094E700BFFA0BFF1F020CFF1FCA
:10A55000EA0BFF1FEC0BFF1FF20BFF1FF00BFF1F9F
:10A560003A13FF1FF80BFF1F0A0CFF1FEE0BFF1F14
:10A57000000CFF1F060CFF1F0E4B1B8807B59BB17D
:10A5800002A8002320F8023D02224FF4886100F067
:10A5900072FABDF80630DB0706D4074B1B7833B1DF
:10A5A0001B210420FFF7CAFC03B05DF804FB034A3B
:10A5B0001370F9E7080CFF1F060CFF1F000CFF1FAC
:10A5C00070B5404D2B780C46002B50D03E4B1B787D
:10A5D00053B100296FD03D4B01221A703C4B1980BA
:10A5E0003C4B00221A8070BD3B4E49B3374B0122D1
:10A5F0001A70374B19803388242B1CD00FD8123B8C
:10A60000934213D93088C0F3071000232B700CB18C
:10A6100040F010002146BDE87040FFF74FBC482BCA
:10A62000F0D101F01CFAFFF71BFCEBE701F00FFA89
:10A6300001F034F8E6E701F00EFAFFF71BFCE1E762
:10A640003088242810D006D8A0F11203012B07D996
:10A6500000F00F00D9E74828FAD101221F4B01E092
:10A660001F4B01221A70F3E701221E4BFAE7174D28
:10A6700079B101232B70164B19801B4B1B7800F00E
:10A680000F0203F00F039A4215DABDE87040FFF79E
:10A6900055BC2B787BB1144B1B7803F00F030C2BAC
:10A6A00005D1124B1B883BB1022000F039FB084A50
:10A6B00000232B70138070BD0D4B1B88002BF6D030
:10A6C0000320F2E7FA0BFF1FEC0BFF1FF20BFF1F3B
:10A6D000F00BFF1F020CFF1FEA0BFF1F060CFF1FF2
:10A6E0003A13FF1F0A0CFF1FED0BFF1FEE0BFF1F9E
:10A6F000FC0BFF1F38B51E4C1E481E4D01220521C4
:10A7000000F0B9F920460222062100F0B4F92388AE
:10A710009B0203F58053238000242B78E0B2834210
:10A7200004F1010421D800F02DFF134B00241C700C
:10A73000124B1C70124B1C70124B1C70124B1C7075
:10A74000124B1C70124B1C80124B1C70124B1C8045
:10A75000124B1C80124B012021461870FFF7AEFBF4
:10A76000104B1C80104B1C7038BD00F0C2FAD4E7AF
:10A77000FE0BFF1F0D0CFF1FEC0BFF1FFA0BFF1F43
:10A78000000CFF1F060CFF1F0A0CFF1F0C0CFF1F05
:10A79000080CFF1FF20BFF1FF00BFF1FF80BFF1F32
:10A7A000ED0BFF1FEA0BFF1F0E0CFF1FF7B53E4F0F
:10A7B00000230124ADF806308DF8054001F03CF986
:10A7C0003A7832B1224640F60E010DF1050000F054
:10A7D00052F900F020FA10F0010F0446334D10D06A
:10A7E0002E7876B94FF490710DF10600012200F039
:10A7F00042F924F0110431469DF80600A4B2FFF797
:10A800009DFBE10611D52B787BB9294B187810F008
:10A8100010010AD120F01003012B06D024F01004FF
:10A8200000F00F00A4B2FFF789FB2B780BB1FFF704
:10A83000E7FD3B7823B39DF8051011F0010105D128
:10A840001B4B187800F00F00FFF778FBA20509D525
:10A85000184800230370184B0122198800F07BF977
:10A8600000F0DEFF9DF8053013F0020F134B1B784C
:10A8700008D04BB100F0CFF9C30501D501F08CF839
:10A8800003B0F0BD002BF5D000F0FCFF9DF80530C3
:10A8900002A803F0020300F8033D012240F60F0175
:10A8A00000F059F9E6E700BF3A13FF1FFA0BFF1F4C
:10A8B000ED0BFF1FF70BFF1F4E13FF1F5813FF1F5A
:10A8C00030B585B00C4615460A460146684603F089
:10A8D000C3F8104900239AB2944210D80E4B0F4A85
:10A8E0001B8814680E490E3BA34294BF9CB2A4B2CD
:10A8F0002246284603F0B0F8204605B030BD1DF8CA
:10A9000003200133581810F8010C9042E3D048F2AC
:10A910000104F1E71C11FF1F4413FF1F1811FF1F53
:10A92000180CFF1F072970B503460D46184915D9A5
:10A93000048844F24530844210D15C8845F241409D
:10A9400084420BD19C8845F24670844206D10B7834
:10A95000A3B11046FEF771FD002070BD0C7884B9DC
:10A960000F2D11D80B4E19462A46304603F074F8C5
:10A97000094BAC551C60094B1C60EDE748F2080020
:10A9800070BD48F2090070BD48F2030070BD00BF01
:10A99000040CFF1F1C11FF1F140CFF1F1811FF1FB9
:10A9A000F8B5134B1B780D461BB1BDE8F840FEF718
:10A9B00045BD104C2368CE18B6F5A06F15D829B147
:10A9C0000A4601460C48184403F046F80B4B1B8816
:10A9D0000E3B9D4214BF0A4B26604FF000001EBF85
:10A9E00020601E6047F6FC70F8BD48F20300F8BD19
:10A9F000040CFF1F140CFF1F180CFF1F5613FF1F22
:10AA00001811FF1F38B50C4B1B6883420D460ED939
:10AA10000A4A0B4914881B1A0E3C9C4228BF1C464C
:10AA200001442246284603F017F8A0B238BD14BFEF
:10AA300048F20400002038BD1811FF1F4413FF1F07
:10AA4000180CFF1F08461146FFF7DCBF10B5064C77
:10AA5000236843B110220021044803F0EBF8044AB4
:10AA600000232360136010BD140CFF1F1C11FF1F77
:10AA70001811FF1F7047F8B506460C46154672B60A
:10AA80000022C1F3471140F20110FEF759FCE1002A
:10AA900041F00601002201F0FE0140F20110FEF734
:10AAA0004FFC210A21F01F01002241F00C0140F26D
:10AAB0000110FEF745FC0022FF2140F20110FEF7D5
:10AAC0003FFC00246F1EAC4201D362B6F8BDBC420D
:10AAD00034BF002201225142C9B240F20110FEF7F8
:10AAE0002FFC30550134EEE7F8B50C461546C1F39E
:10AAF00047110022064640F20110FEF721FCE1005A
:10AB000041F00601002201F0FE0140F20110FEF7C3
:10AB100017FC210A21F01F01002241F00C0140F234
:10AB20000110FEF70DFC0022FF2140F20110FEF79C
:10AB300007FC00246F1EAC4200D3F8BDBC4234BFFA
:10AB4000002201225142C9B240F20110FEF7F8FB87
:10AB500030550134EFE7F8B506460C46154672B697
:10AB60000022C1F3471140F20110FEF7E9FBE100BA
:10AB700041F00601002201F0FE0140F20110FEF753
:10AB8000DFFB210A21F01F01002241F0100140F2F9
:10AB90000110FEF7D5FB00246F1EAC4201D362B654
:10ABA000F8BDBC42315D34BF0022012240F20110E9
:10ABB000FEF7C6FB0134F0E7F8B50C461546C1F3C5
:10ABC00047110022064640F20110FEF7B9FBE100F2
:10ABD00041F00601002201F0FE0140F20110FEF7F3
:10ABE000AFFB210A21F01F01002241F0100140F2C9
:10ABF0000110FEF7A5FB00246F1EAC4200D3F8BD88
:10AC0000BC42315D34BF0022012240F20110FEF748
:10AC100097FB0134F1E738B572B60022114640F2D5
:10AC20000110FEF78DFB00220446022140F20110C4
:10AC3000FEF786FB01220546FF2140F20110FEF7D8
:10AC40007FFB62B644EA052080B238BD002210B511
:10AC5000114640F20110FEF773FB01220446002169
:10AC600040F20110FEF76CFB44EA002080B210BDF8
:10AC700013B5022204464FF401710DF10600FFF7EF
:10AC8000FAFEBDF806300DF106001C4002224FF41A
:10AC90000171ADF80640FFF75EFF02224FF401712B
:10ACA0000248FFF7E8FE02B010BD00BF3411FF1FDD
:10ACB00013B5022204464FF401710DF10600FFF7AF
:10ACC000DAFEBDF806300DF106001C4302224FF4F7
:10ACD0000171ADF80640FFF73EFF02224FF401710B
:10ACE0000248FFF7C8FE02B010BD00BF3411FF1FBD
:10ACF000704737B502AC0122C00004F8012D00F600
:10AD0000070529462046FFF726FF0122294620464F
:10AD1000FFF7B1FE9DF80730DB07F6D503B030BD75
:10AD200037B502AC0023C00004F8013D00F607056A
:10AD3000012229462046FFF70EFF01222946204620
:10AD4000FFF799FE9DF80730DB07F6D403B030BD5E
:10AD500010B5054CC1000822204601F50061FFF73F
:10AD60008AFE204610BD00BF2C11FF1F014B186842
:10AD7000704700BF340BFF1F014B00221A60704761
:10AD8000340BFF1FF8B504460D46164672B6002276
:10AD9000C0F3471140F20120FEF7D2FAE10041F082
:10ADA0000601002201F0FE0140F20120FEF7C8FA80
:10ADB000210A21F01F01002241F00C0140F2012084
:10ADC000FEF7BEFA0022FF2140F20120FEF7B8FA9A
:10ADD00077193446013DBC4201D162B6F8BDA21BD1
:10ADE00095428CBF002201225142C9B240F201209B
:10ADF000FEF7A6FA04F8010BEDE7F8B504460D4698
:10AE0000164672B60022C0F3471140F20120FEF749
:10AE100097FAE10041F00601002201F0FE0140F244
:10AE20000120FEF78DFA210A21F01F01002241F0D6
:10AE3000100140F20120FEF783FA00246F1EAC429D
:10AE400001D162B6F8BDBC42315D34BF002201229F
:10AE500040F20120FEF774FA0134F0E7F8B5044639
:10AE60000D461646C0F34711002240F20120FEF7BE
:10AE700067FAE10041F00601002201F0FE0140F214
:10AE80000120FEF75DFA210A21F01F01002241F0A6
:10AE90000C0140F20120FEF753FA0022FF2140F29C
:10AEA0000120FEF74DFA77193446013DBC4200D12E
:10AEB000F8BDA21B95428CBF002201225142C9B2AB
:10AEC00040F20120FEF73CFA04F8010BEEE7F8B57A
:10AED00004460D461646C0F34711002240F20120F9
:10AEE000FEF72EFAE10041F00601002201F0FE011A
:10AEF00040F20120FEF724FA210A21F01F0100226E
:10AF000041F0100140F20120FEF71AFA00246F1EF2
:10AF1000AC4200D1F8BDBC42315D34BF00220122F9
:10AF200040F20120FEF70CFA0134F1E738B504468F
:10AF30000D4672B60022C0F3471140F20120FEF721
:10AF4000FFF9E10041F00601002201F0FE0140F2AC
:10AF50000120FEF7F5F9210A21F01F01002241F03E
:10AF6000100140F20120FEF7EBF90122294640F2E0
:10AF70000120FEF7E5F962B638BD38B504460D4646
:10AF800072B60022C0F3471140F20120FEF7D8F953
:10AF9000E10041F00601002201F0FE0140F2012033
:10AFA000FEF7CEF9210A21F01F01002241F0100125
:10AFB00040F20120FEF7C4F9E9B2002240F201207C
:10AFC000FEF7BEF90122290A40F20120FEF7B8F986
:10AFD00062B638BD38B504460D4672B60022C0F3DD
:10AFE000471140F20120FEF7ABF9E10041F0060104
:10AFF000002201F0FE0140F20120FEF7A1F9210A32
:10B0000021F01F01002241F0100140F20120FEF763
:10B0100097F9E9B2002240F20120FEF791F9C5F359
:10B020000721002240F20120FEF78AF9C5F307410B
:10B03000002240F20120FEF783F90122290E40F29E
:10B040000120FEF77DF962B638BDF8B504460E461C
:10B05000154672B60022C0F3471140F20120FEF7F8
:10B060006FF9E10041F00601002201F0FE0140F21B
:10B070000120FEF765F9210A21F01F01002241F0AD
:10B08000100140F20120FEF75BF900246F1EAC4274
:10B0900001D162B6F8BDBC42315D34BF002201224D
:10B0A00040F20120FEF74CF90134F0E710B50446F8
:10B0B00072B60022C0F3471140F20120FEF740F9BA
:10B0C000E10041F00601002201F0FE0140F2012002
:10B0D000FEF736F9210A21F01F01002241F00C0190
:10B0E00040F20120FEF72CF90022FF2140F201205E
:10B0F000FEF726F90122FF2140F20120FEF720F998
:10B1000062B610BD37B5254C4FF40043A360FDF780
:10B1100055FF0546FDF752FF401B0028B8BF4042CF
:10B120000428F7DD4FF400436360FDF747FF1C4C34
:10B1300005462369DB0723D50024FDF73FFF0546BD
:10B14000FDF73CFF401B0028B8BF4042B0F5FA7F36
:10B1500021DC02224FF4A0710DF10600FFF78BFCF9
:10B160009DF80630052BEBD14FF43070FFF79EFFB2
:10B1700009214FF43070FFF7D9FE204603B030BDEF
:10B18000FDF71CFF401B0028B8BF4042B0F5FA7F16
:10B19000CFDD0124D1E70124E6E700BF80F00F40B6
:10B1A000C0F00F4010B5044672B60022C0F347113C
:10B1B00040F20120FEF7C4F8E10041F00601002250
:10B1C00001F0FE0140F20120FEF7BAF8210A21F059
:10B1D0001F01002241F00C0140F20120FEF7B0F8FF
:10B1E0000022FF2140F20120FEF7AAF800221146BA
:10B1F00040F20120FEF7A4F801220446FF2140F2AC
:10B200000120FEF79DF862B644EA002080B210BD2E
:10B2100070B5044672B60022C0F3471140F2012017
:10B22000FEF78EF8E10041F00601002201F0FE0178
:10B2300040F20120FEF784F8210A21F01F010022CC
:10B2400041F00C0140F20120FEF77AF80022FF21C4
:10B2500040F20120FEF774F80022114640F201206E
:10B26000FEF76EF800221146064640F20120FEF776
:10B2700067F800221146054640F20120FEF760F80B
:10B2800001220446FF2140F20120FEF759F862B680
:10B29000240444EA0060304340EA052070BDF8B55C
:10B2A00004460E46154672B60022C0F3471140F21E
:10B2B0000120FEF745F8E10041F00601002201F00F
:10B2C000FE0140F20120FEF73BF8210A21F01F01A8
:10B2D000002241F00C0140F20120FEF731F800227B
:10B2E000FF2140F20120FEF72BF877193446013D8B
:10B2F000BC4201D162B6F8BDA21B95428CBF0022B0
:10B3000001225142C9B240F20120FEF719F804F8B7
:10B31000010BEDE738B504460D4672B60022C0F3C6
:10B32000471140F20110FEF70BF8E10041F0060171
:10B33000002201F0FE0140F20110FEF701F8210A9F
:10B3400021F01F01002241F0100140F20110FDF731
:10B35000F7FF0122294640F20110FDF7F1FF62B626
:10B3600038BD38B504460D4672B60022C0F3471109
:10B3700040F20110FDF7E4FFE10041F00601002278
:10B3800001F0FE0140F20110FDF7DAFF210A21F081
:10B390001F01002241F0100140F20110FDF7D0FF23
:10B3A000E9B2002240F20110FDF7CAFF0122290A8A
:10B3B00040F20110FDF7C4FF62B638BD38B504464F
:10B3C0000D4672B60022C0F3471140F20110FDF79E
:10B3D000B7FFE10041F00601002201F0FE0140F25A
:10B3E0000110FDF7ADFF210A21F01F01002241F0FD
:10B3F000100140F20110FDF7A3FFE9B2002240F274
:10B400000110FDF79DFFC5F30721002240F2011056
:10B41000FDF796FFC5F30741002240F20110FDF74A
:10B420008FFF0122290E40F20110FDF789FF62B65D
:10B4300038BD10B5044672B60022C0F3471140F281
:10B440000110FDF77DFFE10041F00601002201F04F
:10B45000FE0140F20110FDF773FF210A21F01F01E8
:10B46000002241F00C0140F20110FDF769FF0022BB
:10B47000FF2140F20110FDF763FF0122FF2140F29E
:10B480000110FDF75DFF62B610BD10B5044672B63F
:10B490000022C0F3471140F20110FDF751FFE10017
:10B4A00041F00601002201F0FE0140F20110FDF71B
:10B4B00047FF210A21F01F01002241F00C0140F258
:10B4C0000110FDF73DFF0022FF2140F20110FDF7C2
:10B4D00037FF0022114640F20110FDF731FF012233
:10B4E0000446FF2140F20110FDF72AFF62B644EA4C
:10B4F000002080B210BD70B5044672B60022C0F3C1
:10B50000471140F20110FDF71BFFE10041F0060179
:10B51000002201F0FE0140F20110FDF711FF210AA7
:10B5200021F01F01002241F00C0140F20110FDF753
:10B5300007FF0022FF2140F20110FDF701FF00226A
:10B54000114640F20110FDF7FBFE002211460646AF
:10B5500040F20110FDF7F4FE00221146054640F2CC
:10B560000110FDF7EDFE01220446FF2140F201101B
:10B57000FDF7E6FE62B6240444EA0060304340EA88
:10B58000052070BD1E4B37B522221A801D4B4FF48B
:10B5900080721A801C4A4FF4805313801B4A138018
:10B5A0001B4B1C4A1A601C4B00241C601B4B02AD39
:10B5B0001C601B4B05F8014D1C601A4B28460122EC
:10B5C00040F60F011C70FFF756FA9DF80730012274
:10B5D00023F0020340F60F0128468DF80730FFF7ED
:10B5E000BAFA114B1C70114B1C70114B1C70114B93
:10B5F0001C70114B1C70114B1C7003B030BD00BF90
:10B600005613FF1F4413FF1F3C13FF1F4E13FF1F52
:10B610005013FF1F3811FF1F5C13FF1F4813FF1F3C
:10B620004013FF1F5813FF1F3A13FF1F3913FF1F4B
:10B630004C13FF1F5513FF1F5413FF1F3813FF1F19
:10B6400038B50020FFF784FB104C4388104D238051
:10B6500003882B800120FFF77BFB0E4A43880E49AD
:10B66000138002880A80288821880144914202DDE3
:10B670001344984207DB0020FFF752FB0120FFF73D
:10B680004FFB002038BD162038BD00BF5613FF1FEA
:10B690003C13FF1F4413FF1F4E13FF1F37B51A4BF8
:10B6A000002420461C70FFF724FB0120FFF721FB3C
:10B6B000164B174A1A60174B1C60174B02AD1C60E3
:10B6C000164B05F8014D1C60154B2846012240F62B
:10B6D0000F011C70FFF7CFF99DF80730012223F00E
:10B6E000020340F60F0128468DF80730FFF733FAC2
:10B6F0000C4B1C700C4B1C700C4B1C700C4B1C70BE
:10B700000C4B1C7003B030BD3A13FF1F5013FF1FCA
:10B710003811FF1F5C13FF1F4813FF1F4013FF1F4B
:10B720005813FF1F3913FF1F4C13FF1F5513FF1F23
:10B730005413FF1F3813FF1F084B1B78012B43794D
:10B7400003D103F00F02042A05D103F00F03042BE9
:10B7500001D1FEF7ADB80220704700BF040CFF1FF7
:10B760002DE9F341254B1B7803F00F03012B804695
:10B770003FD0234B1B78002B3BD0224E3478002C3B
:10B7800039D10788204D0637BAB22988FFF7E3F987
:10B7900002A8012200F8014D40F60D01FFF76BF9F8
:10B7A0009DF807301B070AD4184B29881B881848B6
:10B7B00019440139012289B20470FFF7CCF9154D03
:10B7C0002868804505D080B13A46414602F044F9E8
:10B7D0002868114B1A6852B10022186001232A60B0
:10B7E0003370204602B0BDE8F0814046F1E70B4AD5
:10B7F000F3E7F024F5E70724F3E700BFED0BFF1FA5
:10B800003A13FF1F3913FF1F4E13FF1F4413FF1F6F
:10B81000F70BFF1F5013FF1F4813FF1F3812FF1FA6
:10B82000124B002210B51A70114B124C1A681AB143
:10B83000216809B910490A60104A206812681A6024
:10B8400020B1FFF78DFF0023236010BD0C4A137851
:10B8500053B1590608D523F040031370064BBDE8D9
:10B8600010401868FEF73CB910BD00BF3913FF1F28
:10B870005C13FF1F4013FF1F5013FF1F4813FF1FD0
:10B880005513FF1FF8B50E4B1C6894B10D4D2B7866
:10B8900063B10D4F3E684EB90120FFF72AFA0B4BFA
:10B8A00001201B683B60FFF73BFA2E702046FFF734
:10B8B00057FF074A1378B3FA83F35B091370F8BD97
:10B8C0005C13FF1F3913FF1F4013FF1F4813FF1F97
:10B8D0005813FF1F38B5154B1B7803F00F03012BCE
:10B8E0000C4621D0124D43792A78520704BF012219
:10B8F0002A702A7803F00F03437143EA021343715D
:10B90000FFF72EFF60B144F08004012064B2002CE8
:10B910000BDA084B197804F07F040C431C7038BD17
:10B920002B7801332B70F1E7F02038BDED0BFF1FB2
:10B930003813FF1F5513FF1F10B501884379B1F568
:10B94000807F04464FEA13120DD923F00F03437191
:10B9500001230422C3800823028003810021BDE863
:10B960001040FFF7B7BF0B4B12B11978914210D0BE
:10B9700020461A70FFF7E0FE58B104232380637954
:10B98000208123F00F0363710123E380002120460F
:10B99000E5E710BD5413FF1FF7B5204C02222188A4
:10B9A0000DF10600FFF767F8BDF806301C4A0633B4
:10B9B00011781C4A9BB2ADF8063011B91A490978C2
:10B9C00019B10123137003B0F0BD184F11703A88FC
:10B9D000174D21882868934288BFADF80620BDF82E
:10B9E0000620FFF748F802A8002600F8036D0122A0
:10B9F00040F60501FFF73FF89DF805301B0709D514
:10BA000021883B880B4819440139012289B206700C
:10BA1000FFF731F82868FFF78FFFD4E73C13FF1FCB
:10BA20003913FF1F4C13FF1F5513FF1F5613FF1F22
:10BA30005013FF1FF70BFF1F024B1B780BB1FFF7D3
:10BA4000ABBF70474C13FF1F7047002070470020AA
:10BA5000704700207047002070470020704700208A
:10BA60007047042303800B8000207047014B1B6844
:10BA700003607047A806FF1F014B02685A607047B9
:10BA8000A806FF1F034B5A6812B101321A607047B3
:10BA90001A68FAE7A806FF1FFEE74FF0E023084AFE
:10BAA000C3F8082D074A4CF22053D3814DF62813D2
:10BAB000D381138823F001031B041B0C13807047F0
:10BAC0000080000000200540802800F01F014FF09A
:10BAD00001030F4A04DD8B40C2F88C31D3607047FC
:10BAE000402804DD8B40C2F88831936070472028DD
:10BAF00004DD8B40C2F8843153607047404200F04F
:10BB00001F0058BF41428B40C2F88031136070471C
:10BB100000E100E0802800F01F024FF001030D4912
:10BB200003DD9340C1F88C307047402803DD93401B
:10BB3000C1F888307047202803DD9340C1F8843075
:10BB40007047404200F01F0058BF42429340C1F886
:10BB50008030704700E100E003291ADC202818DC5F
:10BB600042424FF0040302F0030290FBF3F3DBB216
:10BB700000F0030003F1604358BF504203F56443F3
:10BB80008901C0B2C9B2C00001FA00F019680843C7
:10BB900018607047074B1A78D2B2012A02D12229C5
:10BBA00003D15A7001225A7070472129FAD100221C
:10BBB000F7E700BFB006FF1F70B5154611B91B4B64
:10BBC000197070BD022903D1184B01221A7070BD83
:10BBD00004291AD1154B5B78012B25D19488402C70
:10BBE00028BF402400235E1CDBB2A34207D30023FE
:10BBF0001A4602211846BDE8704000F047BF2A6887
:10BC0000D05C00F0C3F83346EDE7032906D1074ABC
:10BC10005378012B08D100239370E9E7052901BF70
:10BC2000024B00221A705A7070BD00BFB006FF1F91
:10BC300010B50446204600F0C1F80028FAD110BD26
:10BC4000704738B50A4C012502460B4600202946AC
:10BC5000A57000F0F5FA224618B10023A370122057
:10BC600038BD937803F0FF00002BFAD138BD00BF38
:10BC7000B006FF1FF8B506460F4600F0F4FC0E4B69
:10BC80001A78012A16D15B78012B13D100F000F944
:10BC900088B10025ECB2A74205D821463046BDE860
:10BCA000F840FFF7CEBF301900F0D6F80135002874
:10BCB000F0D0F2E70C20F8BDB006FF1F08B5402118
:10BCC0000248FFF7D7FF00F095F808BDB306FF1F45
:10BCD00038B5054600F0A8F80B28044609D14021E4
:10BCE0000548FFF7C7FF28B92846BDE8384000F0EF
:10BCF0009BB80024204638BDF306FF1F70B50C46E4
:10BD0000461E00250CB9284670BD16F8010FFFF736
:10BD1000DFFF013C002818BF0B25A4B2F2E738B5BD
:10BD2000451E002415F8010F08B9204638BDFFF75D
:10BD3000CFFF002818BF0B24F4E707B5012300222A
:10BD400000930649064B104600F020FA002814BF65
:10BD50001B20002003B05DF804FB00BFB9BB00004E
:10BD600095BB000038B50C46054600F097F8A04298
:10BD70000AD32C440020A54207D000B138BD15F8E5
:10BD8000010B00F051F8F6E70B2038BD10B50A4A58
:10BD9000117840290ED05378D4180133DBB2402BF0
:10BDA000A07001F101014FF00000117014BF537039
:10BDB000507010BD0B2010BD3307FF1F10B50C4A8B
:10BDC000117891B192F84230D4180133DBB2A478E3
:10BDD0000470402B4FF0000001F1FF31117014BFCF
:10BDE00082F8423082F8420010BD0A2010BD00BF28
:10BDF0003307FF1F014B1878704700BF3307FF1F41
:10BE0000024B1878C0F14000C0B270473307FF1FE3
:10BE1000034B00225A7083F842201A70704700BF0B
:10BE20003307FF1FFFF7F4BF10B50A4A1178402906
:10BE30000ED05378D4180133DBB2402BA07001F13F
:10BE400001014FF00000117014BF5370507010BD0D
:10BE50000B2010BD7607FF1F10B50C4A117891B169
:10BE600092F84230D4180133DBB2A4780470402B2E
:10BE70004FF0000001F1FF31117014BF82F8423021
:10BE800082F8420010BD0A2010BD00BF7607FF1FD8
:10BE9000014B1878704700BF7607FF1F024B1878D8
:10BEA000C0F14000C0B270477607FF1F034B00226D
:10BEB0005A7083F842201A70704700BF7607FF1F40
:10BEC000FFF7F4BF70B50546007801F093F90278EA
:10BED0000023D9B2914207D25C1C03EB83030344D5
:10BEE0005E786B789E4227D1174C2B7A342202FB66
:10BEF0000142D67813B334234B43E218907886423C
:10BF00000CD000F0030204330C2010FB0230211887
:10BF1000205C0B894A68497800F090FBD4F89C308B
:10BF200083B12A46287812F8081F00290CBF032184
:10BF30000521BDE8704018472346CAE793780133CE
:10BF40009370D8E770BD00BFBC07FF1F2DE9F04F0D
:10BF500085B00D4690468DF80F0001F04BF9022D8B
:10BF6000064647D1077800235C1CDBB2BB4210DBDE
:10BF70004FF00009DFF8B0B0CA465FFA89F4A74273
:10BF800012DC284BD3F89C30002B45D105B0BDE81E
:10BF9000F08F03EB830333440DF10F00DA78597807
:10BFA00001F0E2F92346DFE704EB84043444E3784C
:10BFB000A2886178CDF804A0A07800900DF10F0060
:10BFC00001F0B0F9A378032B05D15A4661789DF8AA
:10BFD0000F0001F031FA6178E37841F0100141EA95
:10BFE000C3110022C9B20DF10F0001F0EDF909F102
:10BFF0000109C2E7002DC4D10A490378342000FBAF
:10C0000003138A1C3633294634329A42B9D002F8D7
:10C01000341C02F8331CF7E7424629469DF80F000E
:10C020009847B3E7BC07FF1FC5BE0000F0B40C780B
:10C0300004F06004202C1D4632D14C78042C1DD015
:10C040000AD8012C04D003D3022C20D0032C12D008
:10C0500000202880F0BC7047212C1BD004D8202C55
:10C06000F6D1F0BC00F040B9222C16D0232CEFD131
:10C07000F0BC00F049B9F0BC00F049B902241C80C2
:10C080001468002525701468671C17606570F0BC83
:10C0900000F056B9F0BC00F01FB9F0BC00F076B962
:10C0A000402C06D1044CD4F8A04014B1A446F0BCF6
:10C0B0006047CD20CEE700BFBC07FF1F73B5044625
:10C0C000007801F097F863680093A27A637A43EAF4
:10C0D0000223ADF8043002780023D9B2914207D28E
:10C0E0005D1C03EB830303445E7863789E4225D195
:10C0F000174D237A342202FB0152D67803B334233E
:10C100004B43EA18907886420CD000F003020433C7
:10C110000C2010FB02302918285C0B894A684978EA
:10C1200000F08CFAD5F89C3033B1227A20785AB1DD
:10C1300004F108020521984702B070BD2B46CCE7F8
:10C14000937801339370DAE76A460321F3E700BF7F
:10C15000BC07FF1F07B543680093437A817A43EA1F
:10C160000123ADF80430084BD3F89C3002462BB1C4
:10C17000017A007829B108320521984703B05DF8AB
:10C1800004FB6A460421F8E7BC07FF1F2DE9F843CA
:10C1900005460F461646984601F02CF802789DF8A1
:10C1A000203001328146D2B20021284601F09EF8AB
:10C1B0000446E8B9164A1749284600F086F999F866
:10C1C0000000154B342200FB022209F101011A4440
:10C1D00099463433934201F105010CD1414628467A
:10C1E00000F074F8044618B9C9F89C70C9F8A0604A
:10C1F0002046BDE8F88311F8050C03F8340C11F85B
:10C20000040C03F8330C03F8324C03F8314CE0E72C
:10C210002DC000004DBF0000BC07FF1F08B5074B35
:10C220000022C3F89C20C3F8A02000F0A1F918B99F
:10C23000BDE8084001F06EB808BD00BFBC07FF1F95
:10C240002DE9F041984605460E46174600F0D2FF0C
:10C2500004780023D9B2A14207D2013303EB830251
:10C26000024412F8042CB242F4D1174C34234B434D
:10C27000E218D07892F802E0A0EB0E01C9B20429CE
:10C2800002D1C120BDE8F08100F003010130C0B24D
:10C290004FF00C0C0CFB0133D070A0EB0E001C44D3
:10C2A000C0B2012825716671A760A4F80C8007D17F
:10C2B00043463A4631462846BDE8F04100F0BEB953
:10C2C0000020BDE8F08100BFBC07FF1F014B00202C
:10C2D000196070476008FF1F024B0979197100F05F
:10C2E0008DBF00BF6008FF1F13B5002402AA1C8089
:10C2F000044B42F8041D0979197100F08DFF02B05A
:10C3000010BD00BF6008FF1F00201880704730B4C8
:10C310000C460221198021796488084D012C29716D
:10C3200002D130BC00F08EBF022C02D130BC00F034
:10C3300095BF0020188030BC704700BF6008FF1F09
:10C3400030B40C460221198021796488074D012CF4
:10C35000297102D130BC00F08DBF022C02D130BC5B
:10C3600000F09ABF0020188030BC70476008FF1FA3
:10C37000044B054A19795B791171137203210A2361
:10C38000FFF75EBF6008FF1F0C00FF1FF8B5002716
:10C390001F808B780B4CA371C3F340035A0063F3E7
:10C3A000000206466271FFF7E3FF256845B1A379F5
:10C3B00013F002021ABF3A46222121213046A84733
:10C3C0000020F8BD6008FF1F034B00F108021B6846
:10C3D00000780521184700BF6808FF1F70B5094D98
:10C3E00004462A1D012100F0D7FF802201212046AA
:10C3F00000F0EAFF2B68207800220A21BDE8704097
:10C40000184700BF6808FF1F37B501210DF107026B
:10C41000044600F0C1FF9DF80730074D802B04D182
:10C420002A790121204600F0CFFF2B6820780022D6
:10C430000B21984703B030BD6808FF1F43680521F2
:10C440005A7800F0C1BF73B50122002405460126C9
:10C45000002100F089FF334621468DE8500010226C
:10C46000284600F05FFF22462146284600F07CFF68
:10C47000234621468DE850001022284600F052FF46
:10C4800031460222284600F09FFF32460621284608
:10C4900000F09AFF22469021284600F095FF044BB9
:10C4A00028781B682246214602B0BDE87040184734
:10C4B0006808FF1F42783AB9C178C90141F01001FC
:10C4C00001F0900100F080BF704773B50C468DF805
:10C4D000070001F00DFA1F4D2C600446002836D1EC
:10C4E0001D4A9DF80700102100F0A6FF1B4A0446D4
:10C4F00012219DF8070000F09FFF194A0443142100
:10C500009DF8070000F098FFE4B20443154A9DF837
:10C510000700132100F090FFE4B20443124A9DF893
:10C520000700172100F088FF02AEE4B204430F4A6F
:10C5300016F8010D162100F07FFFE4B20443032238
:10C540000121304600F040FF0323E4B22B71204666
:10C5500002B070BD6808FF1F47C400003DC4000062
:10C56000DDC3000009C40000B5C40000C9C3000059
:10C5700037B502AD174B05F8010D002210212846F2
:10C580001A6000F05BFF12210446284600F056FFB7
:10C5900014210443284600F051FFE4B20443132160
:10C5A000284600F04BFFE4B204431721284600F070
:10C5B00045FFE4B204431621284600F03FFFE4B2F1
:10C5C000204310F0FF0003D19DF8070001F09CF913
:10C5D00003B030BD6808FF1F1FB501218DF80700AB
:10C5E0000DF10E020DF1070000F0D6FE0DF10F0265
:10C5F00006210DF1070000F0CFFE9DF80E30802BD4
:10C6000018D19DF80F309B0714D59DF8070000F056
:10C61000EFFD012804460DD172B60DF1070000F0C0
:10C6200029FB002221460DF107008DF80E2000F0B5
:10C63000CBFE62B69DF80E0004B010BD73B50C467B
:10C6400015461E468DF80700FFF7C6FF802808D064
:10C6500033462A4621460DF1070000F0A7FA02B042
:10C6600070BD0020FBE77047062812D88000012922
:10C67000C0B201D10230C0B2074AC0F34703122151
:10C6800001FB03231A884FF6FF739A4208BFFF206D
:10C690007047FF20704700BF7008FF1F2DE9F04171
:10C6A000314C324D324E4FF0000884F800814FF487
:10C6B000107285F840020F462846FF2101F0BAFAB1
:10C6C0004FF4806241463046C5F8446201F0B2FA48
:10C6D00094F80C3143F0800384F80C3194F80C3159
:10C6E0001B06FBD4234BFF221A7094F80C3143F045
:10C6F000400384F80C31204B196897B341F0004196
:10C700001960194B310AC6F3074201F0FE0183F8A4
:10C710009C1083F8B020320E83F8B420174AC5F875
:10C720004822102283F80821012283F89420BF2296
:10C7300083F8802093F8002102F07F0283F8002123
:10C7400093F8842042F0010283F8842093F8842037
:10C7500042F0100283F8842084221A770020BDE87A
:10C76000F08121F00041CBE7002007407008FF1F57
:10C770000014FF1F1600FF1F007004400016FF1F6B
:10C780000D4B93F80C2102F0BF0283F80C21BF225D
:10C7900083F8802093F8842002F0FE0283F884203E
:10C7A00093F8942002F0FE0283F894201A7F02F09E
:10C7B0007B021A770020704700200740F7B5082356
:10C7C00004248DE81800B1F803300D788878B3F5AB
:10C7D000007F81BF0023CB7002230B71062D71D81F
:10C7E000AB00DCB2012804BF0234E4B24FEA540EBD
:10C7F000354C122707FB0E474FF6FF76B7F800C0FF
:10C80000B4455FD14E78032E5CD801285AD897F8EA
:10C810000FC0BCF1FF0F04BF4FF0000C87F80FC032
:10C82000B1F803C0122101FB0EFE04EB0E0743EA30
:10C830004003BA73FA7B7E7402F0010213435BB2C9
:10C84000D4F84822C7F80220D9B2F9733874D4F862
:10C85000447224F80EC01BB207EBC30E81F0010135
:10C86000CEF80420AEF802C04FF0080E07F833E00F
:10C8700007EBC10ECEF80420AEF802C012FA8CF21B
:10C880004FF0480E07F831E0C4F8482228B917F8ED
:10C89000332062F07F0207F8332002AA02EB800007
:10C8A0002DB20A4950F8082C11F82530012E0CBF82
:10C8B000164642F001063343DBB201F82530002072
:10C8C00003B0F0BD9520FBE77008FF1FC0200740B4
:10C8D000084610B51146FFF7C7FEFF281DD0104BC4
:10C8E0001221C0F3470001FB0030D3F84422C37B80
:10C8F0001CB283F0010312F8341001F07F0102F83A
:10C90000341012F8331001F07F0102F833104FF0A9
:10C91000FF338372C372002010BDC42010BD00BF5E
:10C920007008FF1F73B50C468DF8070011462046AE
:10C930001646FFF799FEFF28054620D021463246CD
:10C940000DF10700FFF7C4FFC5F3470312210D4D9A
:10C9500059436B18D5F848221888121AC5F848228E
:10C9600024B2094A002002F824004FF0FF326A5432
:10C970009A705A70DA701A715A7102B070BD9620AE
:10C98000FBE700BF7008FF1FC02007402DE9F04102
:10C990000E468046114630461746FFF765FE0C4DA1
:10C9A000C0F34700122303FB0050C47BFF2C0DD0C3
:10C9B0003A4631464046FFF78BFF24B2D5F8442271
:10C9C00012F8343063F07B0302F83430BDE8F081B4
:10C9D0007008FF1F10B5084600211446FFF744FEFB
:10C9E000084AC0F34700122101FB0020D2F844326C
:10C9F000C27B03EBC2035A68136823605368636009
:10CA000010BD00BF7008FF1F10B50C462046114630
:10CA1000FFF72AFEFF281AD024B2104B13F8243057
:10CA2000DBB213F00C0F12D09B0712D40C4BD3F8CF
:10CA3000443213F83020D2090DD180F00100C0B289
:10CA400013F83030DB0914BF0320002010BD05208F
:10CA500010BD012010BD032010BD00BFC020074045
:10CA60007008FF1F08B5FFF7FFFD074A1223C0F348
:10CA7000470003FB0020C37BFF2B1EBFD2F84422DC
:10CA8000002102F8331008BD7008FF1F2DE9F041A6
:10CA90000846002190461F46FFF7E6FD2249C0F3F5
:10CAA0004700122404FB0014E57BFF2D39D02288B7
:10CAB0004FF6FF7093B2834233D0D1F8441285F021
:10CAC000010011F9300000282BDB2EB287B901EBF1
:10CAD000C60338465A80D4F802205A6011F835202F
:10CAE00002F0400262F0770201F83620BDE8F081E2
:10CAF00001EBC602BB424FF0000028BF3B466781F6
:10CB0000C4F80680207360735380C2F8048011F863
:10CB1000353003F0400363F0770301F83630BDE8A9
:10CB2000F0819420BDE8F0817008FF1F2DE9F041ED
:10CB30000C460646114620461546FFF795FD194B53
:10CB4000C0F34700122202FB003090F80FE0BEF164
:10CB5000FF0F24D027B2144A6CB1407C012D0CBFCA
:10CB600014211821012818BF41F0010112F82700F3
:10CB7000014302F8271012F827106FF3410102F861
:10CB80002710D3F84432002203F83E203DB92B464B
:10CB90002A4621463046BDE8F041FFF777BFBDE8A1
:10CBA000F08100BF7008FF1FC02007402DE9F04151
:10CBB0000C462046012117469846FFF755FDFF28F1
:10CBC00036D01C4BC0F34700122202FB0030D3F8D2
:10CBD000446290F80FE016F93E30002B28DB23B2B8
:10CBE000154A12F8235015F0020521D10188C0F82A
:10CBF00006701FFA88F242818A42D8BF11460FFAA6
:10CC00008EF206EBC2030573457359805F602CB941
:10CC1000C82306F832302046BDE8F08116F83E30D1
:10CC200003F0400363F0770306F832302C46F2E756
:10CC30009324F0E77008FF1FC0200740034B04480F
:10CC400083F898100122114600F0BEBB0020074077
:10CC5000B00AFF1F054B0648002283F8942080226B
:10CC600083F80C210121FF2200F0AEBB0020074019
:10CC7000B00AFF1F38B51A4C94F8002102F07F0269
:10CC800084F8002194F80C2102F0DF0284F80C21D2
:10CC900094F8802042F0200284F8802094F88420C8
:10CCA00002F0DF0284F8842094F8942002F0DF027E
:10CCB00084F8942094F8942042F0040284F894209C
:10CCC00044F62065013DADB200F0BCFE002DF9D167
:10CCD00094F8943003F0FB0384F8943038BD00BF1F
:10CCE000002007402DE9F04FD84DD94C95F88070C1
:10CCF00095F8843095F8906087B0FF221F4094F833
:10CD000040328DF809208DF80C308DF80D2000236D
:10CD100001210DF1090204F510708DF80E30049315
:10CD20008DF815308DF816308DF80F308DF81430E1
:10CD300000F032FB95F80C31D907F6B20FD59DF80B
:10CD40000930802B0BD195F8003103F07F0385F873
:10CD5000003195F80C3103F0DF0385F80C317A07C8
:10CD600011D5BA4B042093F8A41093F8A02083F8AF
:10CD7000800006AB42EA012223F80E2D03A91220FF
:10CD8000049300F06DFBFB074BD5B04DB048012379
:10CD9000BF2685F8803085F8886095F894300027A4
:10CDA00043F0020385F894304FF4107285F89870C0
:10CDB000FF2185F8007100F03DFF4FF48062394695
:10CDC000D4F8440200F036FFD4F8443203F500737F
:10CDD000C4F848329F4BFF221A7095F8943003F044
:10CDE000FD0385F8943095F80C3143F0400385F845
:10CDF0000C319F2385F88C6085F8843095F8943049
:10CE000003F0DF0385F8943003A9102000F028FB1D
:10CE100095F8943003F0DF0385F8943007B0BDE84F
:10CE2000F08F3D0740F19380884B082283F88020E3
:10CE30003309C6F3C000062B8DF80D308DF80F00B6
:10CE400000F2F480C6F3800202EB830208B10232E2
:10CE5000D2B2D4F8446206EBC201C2F34705D1F85E
:10CE600004E04988ADF81510122101FB0541CDF809
:10CE700010E091F80FC08CF0010C81F80FC016F88B
:10CE8000321082F0010A5FFA8AFAC1F380110FFAB8
:10CE90008AF881F00101890106EBC80906F838100B
:10CEA000002800F0D980DFF8ACB19BB99BF80020D6
:10CEB00082B9FF2219468BF8002003A81A46019375
:10CEC000FFF706FD019B06F838301A46194603A8FD
:10CED000FFF7DCFD9BF80030012B04D09DF80D30EE
:10CEE000002B00F0AD80122101FB0541BDF81500BB
:10CEF0008B894A8903449BB293428B8109D3B1F851
:10CF000000E0C0B2864540F09380897B012940F063
:10CF10008F80122101FB0544D4F8061020881944A3
:10CF2000D31A8342D8BF98B2A9F80200C9F80410F6
:10CF300016F83A3003F0400363F0770306F8383010
:10CF4000424A92F8943003F0DF0382F89430B80735
:10CF500017D53E4C022384F8803094F8883094F83A
:10CF60008C2003A9134016208DF8143000F078FAB5
:10CF7000BF2384F8883094F8943003F0DF0384F8FA
:10CF80009430F9061CD5314C202384F880301023CE
:10CF900084F8803003A9142000F062FA94F80C3170
:10CFA00043F0200384F80C3194F8003143F08003FF
:10CFB00084F8003194F8843043F0200384F88430FE
:10CFC000BA060DD5214C202384F8803003A9132004
:10CFD00000F046FA94F8843003F0DF0384F88430DC
:10CFE0003B067FF51BAF0DF10A02FF23102103A8BA
:10CFF0008DF80D3000F0D0F99DF80A30134C012B5C
:10D0000004BF8DF80F3000224FF0800308BF8DF869
:10D010000D2003A984F88030172000F021FA94F83D
:10D02000943003F0DF0384F89430F7E6FF2210E732
:10D03000122202FB0544D4F806200492ADF8153004
:10D0400003A99DF80D0000F00BFA79E700200740D6
:10D050007008FF1F1600FF1F6BB916F832202F490A
:10D0600002F03C02342A35D101238DF80E309EF8AF
:10D070000030DB090B70122101FB05414FF6FF73F5
:10D080004A899A42DCD0BDF815E08B8973449BB283
:10D090008B8109888E4501D19A420CD88AB3B2FBA4
:10D0A000F1F001FB102080B258BB122000FB0540BC
:10D0B000807B012825D1D21A8A42D8BF91B2122290
:10D0C00002FB0544C9B9D4F80230C9F80430A9F804
:10D0D00002102DE70A78012ACDD1FF2008701946E9
:10D0E00003A80193FFF7F4FB019B06F838301A46BA
:10D0F000194603A8FFF7CAFCBDE7D4F8062013447D
:10D10000E3E7122202FB0544D4F80620ADF81530FF
:10D110004FF0FF330492A372E37291E71600FF1FF2
:10D1200013460A46194600F085BD00BF30B50329F5
:10D13000039C04981DD12BB9164A22600422028058
:10D14000002030BD40F209418B420FD1022A4FF03E
:10D1500000030CD810490C2505FB0313D9681B6983
:10D1600051F8221021609B5C0380E9E70123012232
:10D17000F0E7072901D9CD2030BD074B03EB810231
:10D18000126A2260002AF6D003EB4103B3F8403064
:10D19000EAE700BF1700FF1F10DE000001299FBF54
:10D1A000034B5B5C1370002088BFCD20704700BF2D
:10D1B000BC0AFF1F01299DBF024B00205A54CD20FD
:10D1C000704700BFBC0AFF1F19B14B1E584258419F
:10D1D000704701207047054B1A788A4204D058786E
:10D1E000431A58425841704701207047BC0AFF1F3C
:10D1F000002070470048704760DE000001299FBF93
:10D20000044BC1EBC101C918002094BF1160CD20AF
:10D21000704700BF1B00FF1F012930B50ED8084D15
:10D22000C1EBC10108231068C45CC818284401334D
:10D230000F2B00F8084CF6D1002030BDCD2030BDBA
:10D240001B00FF1F01299FBF034B03EB410100207F
:10D25000116088BFCD207047BE0AFF1F01299FBF04
:10D26000034B03EB41010020116088BFCD207047C4
:10D27000C20AFF1F01290AD813681878054B03EB6F
:10D280004101887013685B78CB7000207047CD2017
:10D29000704700BFBC0AFF1F01290AD8136818781D
:10D2A000054B03EB4101887113685B78CB7100205B
:10D2B0007047CD20704700BFBC0AFF1F084B5A784B
:10D2C00003F8022BFF210022D1540132072AFBD19F
:10D2D000044A0023052199540133072BFBD17047E1
:10D2E000C60AFF1FCF0AFF1F00BF7047013AD2B224
:10D2F000062A10B51C4608D8054B5A70FFF7DEFF0A
:10D300002146BDE81040FFF7C9B9992010BD00BF04
:10D31000C60AFF1F024B00225A70FFF731BA00BF46
:10D32000C60AFF1F37B50F4C257805B9C1B98DF86E
:10D3300002308DF800109DF81830ADF803206946D2
:10D340009DF81C2000788DF80130FFF737FA9DF822
:10D3500000301BB110B92378013B237003B030BDFE
:10D360009520FBE7C60AFF1F38B50A4B0D461C780F
:10D3700059788C421C4600D14DB929460078FFF7F8
:10D38000D1FA2DB120B923780133237038BD96200E
:10D3900038BD00BFC60AFF1F4B1E062B05D8094B20
:10D3A00019444B78137000207047CB0607D501F065
:10D3B0000F01062903D8034B19444B7AF2E7822068
:10D3C000704700BFC60AFF1F4B1E062B2DE9F04118
:10D3D0008046174605D8174B19444A700020BDE80F
:10D3E000F081CB0622D501F00F05062D1ED8012AAB
:10D3F0004FEAD1140F4E06D122462946FFF7C6FA4E
:10D4000035446F72EAE7002AFAD173195B7A012B6F
:10D41000F6D122462946FFF789FB002DF0D184F092
:10D42000010229464046FFF781FBE9E78220BDE87B
:10D43000F08100BFC60AFF1F00207047062903D9EC
:10D44000A1F11003072B07D8044B53F82130002B10
:10D450000CBFC42000207047C420704788DE000045
:10D46000102810B50C4601D1FFF728FF034B53F8E5
:10D4700020300BB120469847002010BD88DE000008
:10D480001FB5144602228DF807001A8005210DF100
:10D490000F020DF10700FFF77FFF034B9DF80F20F0
:10D4A0001A80236004B010BDD80AFF1F1FB51446B0
:10D4B00001228DF807001A8004210DF10F020DF1F1
:10D4C0000700FFF769FF044B9DF80F201A8000202A
:10D4D000236004B010BD00BFD80AFF1FF0B50026BE
:10D4E00085B01E8049888DF80700ADF80E10FFF753
:10D4F0006BFE18B3BDF80E20114F04ACB2FA82F2E5
:10D50000520901210DF10700FFF75EFF34F8022DEB
:10D510000421D2B20DF10700FFF756FF7B682246C7
:10D52000012105469DF8070098477B689DF8070094
:10D53000324602219847284605B0F0BD0425FAE797
:10D54000D80AFF1F73B502AC002504F8010D0E4682
:10D550001D80042201212046FFF736FF7288024B0E
:10D5600028461A7202B070BDD80AFF1F13B54C8846
:10D5700089888DE80C000B46E2B2210AFFF7D6FD40
:10D5800002B010BD2DE9F04186B017461E4606AA2E
:10D5900000238846059303238DF80F0002F8083D09
:10D5A00001210DF10F00FFF7F7FE98F80050274C0E
:10D5B00015F0030528D10DF1110206210DF10F0020
:10D5C000FFF7EAFE9DF811309DF80F0003F003030A
:10D5D00023800DF11203019305AB00932A462B46DD
:10D5E0000221FFF7A3FD059BDB7913F0400F238891
:10D5F00014BF43F0010323F001032380022333808F
:10D600003C6006B0BDE8F081012D08D19DF81030D6
:10D61000012B02D198F80430ABB90023EDE7022DBD
:10D62000EED198F8041041F010010DF11202C9B2C8
:10D630000DF10F00FFF7B0FE9DF8123003F001036B
:10D6400023803580DCE7CD20DAE700BFD80AFF1F52
:10D650007FB500221A800B784E788DF8070013F002
:10D6600003030D46C6F3400634D1FEB14B88013B9F
:10D670009BB2012B52D80DF10F0206210DF10700CC
:10D68000FFF78AFE044670B9AB7801229A409DF8F4
:10D690000F301A43D2B206210DF107008DF80F208A
:10D6A000FFF792FE0446204604B070BD4E88012E5E
:10D6B00034D10DF10F0206210DF10700FFF76CFECA
:10D6C00004460028EFD1AA7896409DF80F2022EA60
:10D6D0000602E0E7022B21D109798DF80F103246BE
:10D6E00041F010010DF10700FFF76EFE6B78002E80
:10D6F00014BF07210821012B044607D19DF80F0014
:10D70000C10900F00F00FFF7ADF90821044B9DF8A7
:10D7100007005B680DF10F029847C4E7CD24C2E70C
:10D72000D80AFF1F10B500241C800B7803F00303F8
:10D73000012B05D18A780979FFF73CFD204610BD01
:10D74000042010BD38B515460A7802F00302012AFC
:10D7500007D1054C1A8009792246FFF71FFD2C607E
:10D7600038BD042038BD00BFD80AFF1F13B5CD292E
:10D770008DF8070007D1012290210DF10700FFF776
:10D7800023FE02B010BD0D491C88088A126884422D
:10D7900088BF18800C461B889DF807000021FEF703
:10D7A0004DFF94F90A30002BEBDA00231A46194694
:10D7B0000DF10700FFF76AF9E3E700BFD80AFF1F82
:10D7C00073B5054600266A4601218DF80060019672
:10D7D000FFF7E2FDAA78434C012A52D1686803683A
:10D7E000C4F80A304368A07AC4F80E3004F10A0184
:10D7F00010F0600F1ED1E27A3B4B53F82240002C10
:10D800003DD09DF80000022839D802EB42021344B3
:10D81000034493F83430012B31D10DF1020301AAF6
:10D820002878A0470DF1020301AA01462878FFF7E6
:10D830009DFF13E0238AADF80230202B17D87BB16F
:10D8400002060DD40A68C4F812204A68C4F81620EB
:10D85000314604F11A022846FFF718F902B070BDEC
:10D86000E46B64B10DF1020301AA2049D8E702A8D4
:10D870002B7800F8073D9021FFF7A6FDEEE7CD20BD
:10D88000D0E79DF80030042B10D12B78217A02AD1F
:10D8900005F8063D2846FFF7D1F901221146284632
:10D8A000FFF792FD227A03212846E5E794F90A3032
:10D8B000002BD3DBEB78002BD0D1E66B86B1B5F82B
:10D8C000093028780833ADF8023004F112010DF167
:10D8D000020301AAB04701460DF1020301AAA5E720
:10D8E000CD21F9E7D80AFF1FE8DE0000E20AFF1F9A
:10D8F000034B5960DA630021024AFFF79DBD00BF68
:10D90000D80AFF1FC1D7000007B502AB054A03F8CC
:10D91000010D002118465160D163FFF78FFD03B060
:10D920005DF804FBD80AFF1F00207047354B41F219
:10D9300048015A5822F00F0242F002025A5041F2B6
:10D9400004015A5842F480225A5041F234015A5884
:10D9500042F480225A5003F52C33602193F894202E
:10D9600042F0020283F89420C02283F80021FF22B3
:10D970001A7483F8802083F8882083F8842000229A
:10D9800083F88C2083F80C111F491A75080A00F0DF
:10D99000FE0083F8982083F8C02083F8C42083F821
:10D9A000C82083F8CC2083F8D02083F8D42083F8D3
:10D9B000D82083F8DC2083F8E02083F8E42083F883
:10D9C000E82083F8EC2083F8F02083F8F42083F833
:10D9D000F82083F8FC2083F89C00C1F30740090E6F
:10D9E00083F8B00083F8B41083F8AC201A7783F87A
:10D9F000082193F8942002F0D40242F0010283F847
:10DA000094207047007004400014FF1F024B4FF435
:10DA100000729A60704700BF00E100E0034B4FF4D2
:10DA20000072C3F888219A60704700BF00E100E0EF
:10DA300008B5FEF782F910B9FFF7F0FF08BD1B200B
:10DA400008BD00BF034B4AF202629A814BF280424A
:10DA50009A81704700200540844641EA000313F094
:10DA600003036DD1403A41D351F8043B40F8043BE5
:10DA700051F8043B40F8043B51F8043B40F8043BA8
:10DA800051F8043B40F8043B51F8043B40F8043B98
:10DA900051F8043B40F8043B51F8043B40F8043B88
:10DAA00051F8043B40F8043B51F8043B40F8043B78
:10DAB00051F8043B40F8043B51F8043B40F8043B68
:10DAC00051F8043B40F8043B51F8043B40F8043B58
:10DAD00051F8043B40F8043B51F8043B40F8043B48
:10DAE00051F8043B40F8043B403ABDD2303211D3E8
:10DAF00051F8043B40F8043B51F8043B40F8043B28
:10DB000051F8043B40F8043B51F8043B40F8043B17
:10DB1000103AEDD20C3205D351F8043B40F8043BE7
:10DB2000043AF9D2043208D0D2071CBF11F8013BE5
:10DB300000F8013B01D30B8803806046704700BFAB
:10DB4000082A13D38B078DD010F003038AD0C3F1BA
:10DB50000403D21ADB071CBF11F8013B00F8013B9C
:10DB600080D331F8023B20F8023B7BE7043AD9D35B
:10DB7000013A11F8013B00F8013BF9D20B78037030
:10DB80004B7843708B78837060467047FDF785FF54
:10DB9000002103E00A4B5B584350043109480A4B0B
:10DBA00042189A42F6D3094A02E000231360043275
:10DBB000074B9A42F9D300F00DF8804770470000F8
:10DBC00074DF00000800FF1F2C05FF1F0006FF1F69
:10DBD0002418FF1F10B5FAF754FCFAF7BBFCFBF74B
:10DBE000C5FAFBF7D5FAFBF7DFF9FBF73DFB0020A1
:10DBF000FBF7EAF90020FBF757FAFBF713FBFDF7F9
:10DC000081FAC4B20CB9FBF70BFDFAF7DFFCFBF7A6
:10DC100055F8074B02224CB19A60FAF7EDFCFBF77E
:10DC20004EF8002CF9D1FBF71BFDF6E75A60F4E73C
:10DC300000F00F4070B4860746D0541E002A41D031
:10DC4000CAB2034602E014F1FF343BD303F8012BC0
:10DC50009D07F8D1032C2ED9CDB245EA05250F2C0E
:10DC600045EA054519D903F110022646103E0F2E4C
:10DC700042F8105C42F80C5C42F8085C42F8045C24
:10DC800002F11002F2D8A4F1100222F00F0204F007
:10DC90000F041032032C13440DD91E462246043AB9
:10DCA000032A46F8045BFAD8221F22F0030204324A
:10DCB000134404F003042CB1C9B21C4403F8011B43
:10DCC0009C42FBD170BC704714460346C2E700BFBC
:10DCD000024B13B1024800F005B870470000000085
:10DCE000F1DC0000002301461A46184600F01EB879
:10DCF00038B50A4C0A4D641BA4100AD004F18043C5
:10DD0000013B05EB8305013C55F804399847002C8D
:10DD1000F9D1BDE8384000F021B900BF74DF000040
:10DD200070DF0000704700BF704700BF2DE9F84367
:10DD30002C4D0646286898460F469146FFF7F2FF9D
:10DD4000294B1C68D4F84831002B3ED05A681F2A52
:10DD50001CDC02F1010E76B103EB82010124C1F853
:10DD60008890D3F8880194402043022EC3F888019C
:10DD7000C1F8088123D00232C3F804E0286843F8D0
:10DD80002270FFF7D1FF0020BDE8F883174B0BB3DB
:10DD90004FF4C870AFF300800346D8B1D4F84821DF
:10DDA0000260002141600A46C4F848014FF0010EAC
:10DDB000C0F88811C0F88C11002EDCD0CCE7D3F865
:10DDC0008C110C43C3F88C41D5E704F5A673C4F855
:10DDD0004831BBE72868FFF7A7FF4FF0FF30BDE8E9
:10DDE000F88300BF2805FF1F4CDF00000000000083
:10DDF0008025000040380000004B000080700000CB
:10DE00000096000000E10000002C010000C20100AB
:10DE10001700FF1F040000000904000074DE00006A
:10DE200084DE000000000000000000000000000090
:10DE300000000000EE00FF1FAB00FF1F000000000D
:10DE400000000000000000000000000000000000D2
:10DE5000000012004300000000000000000000006D
:10DE60000301020110000202001000030301100070
:10DE7000000100001700FF1F7100FF1F4B00FF1F74
:10DE80002900FF1F043A2622C1D70000BDC00000B0
:10DE900055C10000C5BE0000E9D20000E9D2000073
:10DEA000E9D20000E9D20000E9D20000E9D2000086
:10DEB000E9D20000E9D20000E9D20000E9D2000076
:10DEC000E9D20000E9D2000047C40000DDC3000031
:10DED0003DC4000009C40000DDC30000E9D2000019
:10DEE000C9C30000B5C4000085D5000051D60000AC
:10DEF0000000000051D600000000000045D50000E1
:10DF00006DD5000000000000ADD40000DDD400009D
:10DF100045D7000025D7000081D400000101000191
:10DF200001000000000101000000000001010101EA
:10DF300001000000010100010100010000010000DA
:10DF40000100003030313256313030000001FF1F07
:10DF5000F8B500BFF8BC08BC9E467047F8B500BFD6
:08DF6000F8BC08BC9E467047A6
:08DF6800D1DC0000358400004B
:04DF70001184000018
:10DF740043DF0000A1200000000002000000FF04B5
:10DF840003090400C20100000008000000000000B2
:10DF94000022034200410044002000530054005278
:10DFA4000049004E004700200049004E004400454F
:10DFB40000580026034500760061006C007500617E
:10DFC40000740069006F006E002000440065007654
:10DFD4000069006300650020003A035400520049C0
:10DFE400004E0041004D004900430020004D006FE9
:10DFF40000740069006F006E00200043006F006E23
:10E0040000740072006F006C0020002000200020CB
:10E0140000200009024300020100C032090400008C
:10E02400010202000005240010010524010101047D
:10E0340024020605240600010705830310000A09CB
:10E04400040100020A000000070581021000000715
:10E0540005020210000012010002020000103C2A16
:10E06400000702000102000100000000EC03FF1F92
:10E074005404FF1FBC04FF1F000000000000000048
:10E08400000000000000000000000000000000008C
:10E09400000000000000000000000000000000007C
:10E0A400000000000000000000000000000000006C
:10E0B400000000000000000000000000000000005C
:10E0C400000000000000000000000000000000004C
:10E0D400000000000000000000000000000000003C
:10E0E400000000000000000000000000000000002C
:10E0F400000000000000000000000000000000001C
:10E10400000000000000000000000000000000000B
:10E1140001000000000000000E33CDAB34126DE6A8
:10E12400ECDE05000B000000000000000000000011
:10E1340000000000000000000000000000000000DB
:10E1440000000000000000000000000000000000CB
:10E1540000000000000000000000000000000000BB
:10E1640000000000000000000000000000000000AB
:04E494000018FF1F4E
:10E4980074DF00000800FF1F2405000000000000D2
:08E4A80000000000000000006C
:040000030000DB8D91
:00000001FF
